Archive member included because of file (symbol)

board/ami/libami.a(lowlevel_init.o)
                              cpu/arm920t/start.o (lowlevel_init)
cpu/arm920t/libarm920t.a(interrupts.o)
                              cpu/arm920t/start.o (do_undefined_instruction)
cpu/arm920t/s3c24x0/libs3c24x0.a(interrupts.o)
                              cpu/arm920t/libarm920t.a(interrupts.o) (reset_cpu)
cpu/arm920t/s3c24x0/libs3c24x0.a(speed.o)
                              cpu/arm920t/s3c24x0/libs3c24x0.a(interrupts.o) (get_PCLK)
lib_arm/libarm.a(_udivsi3.o)  cpu/arm920t/s3c24x0/libs3c24x0.a(interrupts.o) (__udivsi3)
lib_arm/libarm.a(board.o)     cpu/arm920t/s3c24x0/libs3c24x0.a(speed.o) (hang)
lib_arm/libarm.a(div0.o)      lib_arm/libarm.a(_udivsi3.o) (__div0)
net/libnet.a(net.o)           lib_arm/libarm.a(board.o) (copy_filename)
net/libnet.a(tftp.o)          net/libnet.a(net.o) (TftpStart)
net/libnet.a(bootp.o)         net/libnet.a(net.o) (BootpRequest)
net/libnet.a(rarp.o)          net/libnet.a(net.o) (RarpRequest)
net/libnet.a(eth.o)           lib_arm/libarm.a(board.o) (eth_initialize)
net/libnet.a(nfs.o)           net/libnet.a(net.o) (NfsStart)
drivers/libdrivers.a(cs8900.o)
                              lib_arm/libarm.a(board.o) (cs8900_get_enetaddr)
common/libcommon.a(main.o)    lib_arm/libarm.a(board.o) (main_loop)
common/libcommon.a(cmd_autoscript.o)
                              (__u_boot_cmd_autoscr)
common/libcommon.a(cmd_bdinfo.o)
                              (__u_boot_cmd_bdinfo)
common/libcommon.a(cmd_boot.o)
                              (__u_boot_cmd_reset)
common/libcommon.a(cmd_bootm.o)
                              (__u_boot_cmd_imls)
common/libcommon.a(cmd_cache.o)
                              (__u_boot_cmd_dcache)
common/libcommon.a(cmd_console.o)
                              (__u_boot_cmd_coninfo)
common/libcommon.a(cmd_date.o)
                              (__u_boot_cmd_date)
common/libcommon.a(cmd_elf.o)
                              (__u_boot_cmd_bootvx)
common/libcommon.a(cmd_flash.o)
                              (__u_boot_cmd_protect)
common/libcommon.a(cmd_itest.o)
                              (__u_boot_cmd_itest)
common/libcommon.a(cmd_load.o)
                              (__u_boot_cmd_loady)
common/libcommon.a(cmd_mem.o)
                              (__u_boot_cmd_mtest)
common/libcommon.a(cmd_misc.o)
                              (__u_boot_cmd_sleep)
common/libcommon.a(cmd_net.o)
                              (__u_boot_cmd_nfs)
common/libcommon.a(cmd_nvedit.o)
                              (__u_boot_cmd_run)
common/libcommon.a(command.o)
                              (__u_boot_cmd_question_mark)
common/libcommon.a(console.o)
                              cpu/arm920t/libarm920t.a(interrupts.o) (printf)
common/libcommon.a(devices.o)
                              common/libcommon.a(cmd_console.o) (stdio_names)
common/libcommon.a(dlmalloc.o)
                              common/libcommon.a(cmd_autoscript.o) (free)
common/libcommon.a(env_common.o)
                              common/libcommon.a(cmd_nvedit.o) (env_get_char)
common/libcommon.a(env_flash.o)
                              common/libcommon.a(env_common.o) (env_ptr)
common/libcommon.a(exports.o)
                              lib_arm/libarm.a(board.o) (jumptable_init)
common/libcommon.a(flash.o)   common/libcommon.a(cmd_load.o) (addr2info)
common/libcommon.a(lists.o)   common/libcommon.a(devices.o) (ListCreate)
common/libcommon.a(s_record.o)
                              common/libcommon.a(cmd_load.o) (srec_decode)
common/libcommon.a(xyzModem.o)
                              common/libcommon.a(cmd_load.o) (xyzModem_stream_open)
common/libcommon.a(crc16.o)   common/libcommon.a(xyzModem.o) (cyg_crc16)
lib_generic/libgeneric.a(crc32.o)
                              common/libcommon.a(cmd_autoscript.o) (crc32)
lib_generic/libgeneric.a(display_options.o)
                              lib_arm/libarm.a(board.o) (print_size)
lib_generic/libgeneric.a(string.o)
                              net/libnet.a(net.o) (strcpy)
lib_generic/libgeneric.a(vsprintf.o)
                              lib_arm/libarm.a(board.o) (simple_strtoul)
lib_generic/libgeneric.a(zlib.o)
                              common/libcommon.a(cmd_bootm.o) (inflateEnd)
lib_generic/libgeneric.a(ctype.o)
                              lib_generic/libgeneric.a(vsprintf.o) (_ctype)
board/ami/libami.a(ami.o)     lib_arm/libarm.a(board.o) (board_init)
board/ami/libami.a(flash.o)   lib_arm/libarm.a(board.o) (flash_init)
cpu/arm920t/libarm920t.a(cpu.o)
                              lib_arm/libarm.a(board.o) (cpu_init)
cpu/arm920t/s3c24x0/libs3c24x0.a(serial.o)
                              common/libcommon.a(cmd_load.o) (serial_setbrg)
lib_arm/libarm.a(_divsi3.o)   common/libcommon.a(cmd_date.o) (__divsi3)
lib_arm/libarm.a(_modsi3.o)   net/libnet.a(nfs.o) (__modsi3)
lib_arm/libarm.a(_umodsi3.o)  net/libnet.a(tftp.o) (__umodsi3)
lib_arm/libarm.a(armlinux.o)  common/libcommon.a(cmd_bootm.o) (do_bootm_linux)
lib_arm/libarm.a(cache.o)     common/libcommon.a(cmd_elf.o) (flush_cache)
rtc/librtc.a(date.o)          common/libcommon.a(cmd_date.o) (GregorianDay)
rtc/librtc.a(s3c24x0_rtc.o)   common/libcommon.a(cmd_date.o) (rtc_get)

Memory Configuration

Name             Origin             Length             Attributes
*default*        0x00000000         0xffffffff

Linker script and memory map

                0x00000000                . = 0x0
                0x00000000                . = ALIGN (0x4)

.text           0x33f80000    0x11f18
 cpu/arm920t/start.o(.text)
 .text          0x33f80000      0x400 cpu/arm920t/start.o
                0x33f80048                _bss_start
                0x33f8004c                _bss_end
                0x33f80044                _armboot_start
                0x33f80000                _start
 *(.text)
 .text          0x33f80400       0x64 board/ami/libami.a(lowlevel_init.o)
                0x33f80404                lowlevel_init
 .text          0x33f80464      0x260 cpu/arm920t/libarm920t.a(interrupts.o)
                0x33f8067c                do_fiq
                0x33f805c8                do_undefined_instruction
                0x33f8048c                show_regs
                0x33f806a0                do_irq
                0x33f80470                bad_mode
                0x33f80610                do_prefetch_abort
                0x33f80468                disable_interrupts
                0x33f80658                do_not_used
                0x33f80634                do_data_abort
                0x33f805ec                do_software_interrupt
                0x33f80464                enable_interrupts
 .text          0x33f806c4      0x25c cpu/arm920t/s3c24x0/libs3c24x0.a(interrupts.o)
                0x33f807f8                set_timer
                0x33f80774                reset_timer
                0x33f806c4                interrupt_init
                0x33f808f4                get_tbclk
                0x33f807e4                get_timer
                0x33f80744                reset_timer_masked
                0x33f80778                get_timer_masked
                0x33f80808                udelay
                0x33f80864                udelay_masked
                0x33f80900                reset_cpu
                0x33f808e0                get_ticks
 .text          0x33f80920       0xc0 cpu/arm920t/s3c24x0/libs3c24x0.a(speed.o)
                0x33f80988                get_HCLK
                0x33f809b0                get_PCLK
                0x33f80980                get_FCLK
                0x33f809d8                get_UCLK
 .text          0x33f809e0       0x98 lib_arm/libarm.a(_udivsi3.o)
                0x33f809e0                __udivsi3
 .text          0x33f80a78      0x2fc lib_arm/libarm.a(board.o)
                0x33f80b60                hang
                0x33f80b70                start_armboot
                0x33f80a78                sbrk
 .text          0x33f80d74        0x4 lib_arm/libarm.a(div0.o)
                0x33f80d74                __div0
 .text          0x33f80d78     0x129c net/libnet.a(net.o)
                0x33f81b24                getenv_IPaddr
                0x33f813dc                NetCksumOk
                0x33f80f90                NetSetTimeout
                0x33f81444                copy_filename
                0x33f81400                NetEthHdrSize
                0x33f81498                ip_to_string
                0x33f8105c                ArpTimeoutCheck
                0x33f81514                NetReceive
                0x33f81aa4                string_to_ip
                0x33f81274                NetSendUDPPacket
                0x33f814f0                print_IPaddr
                0x33f80d78                NetSetEther
                0x33f81c00                NetLoop
                0x33f80e38                ArpRequest
                0x33f81b34                VLAN_to_string
                0x33f81be8                getenv_VLAN
                0x33f810e8                NetCksum
                0x33f81134                NetSetIP
                0x33f81b90                string_to_VLAN
                0x33f80fdc                NetStartAgain
                0x33f80fcc                NetSetHandler
                0x33f810e4                NetSendPacket
 .text          0x33f82014      0x6b8 net/libnet.a(tftp.o)
                0x33f824a8                TftpStart
 .text          0x33f826cc      0x65c net/libnet.a(bootp.o)
                0x33f82a7c                BootpRequest
 .text          0x33f82d28      0x1a0 net/libnet.a(rarp.o)
                0x33f82d80                RarpRequest
 .text          0x33f82ec8        0x8 net/libnet.a(eth.o)
                0x33f82ec8                eth_initialize
 .text          0x33f82ed0      0xefc net/libnet.a(nfs.o)
                0x33f83b70                NfsStart
 .text          0x33f83dcc      0x5b4 drivers/libdrivers.a(cs8900.o)
                0x33f840e0                eth_halt
                0x33f83f18                cs8900_get_enetaddr
                0x33f842f4                cs8900_e2prom_read
                0x33f84328                cs8900_e2prom_write
                0x33f84184                eth_rx
                0x33f84100                eth_init
                0x33f84208                eth_send
 .text          0x33f84380      0x900 common/libcommon.a(main.o)
                0x33f84640                run_command
                0x33f84c04                do_run
                0x33f8445c                readline
                0x33f84a90                main_loop
 .text          0x33f84c80      0x260 common/libcommon.a(cmd_autoscript.o)
                0x33f84ea0                do_autoscript
                0x33f84c80                autoscript
 .text          0x33f84ee0       0xe4 common/libcommon.a(cmd_bdinfo.o)
                0x33f84ef4                do_bdinfo
 .text          0x33f84fc4       0x88 common/libcommon.a(cmd_boot.o)
                0x33f84fc4                do_go
 .text          0x33f8504c      0xfe8 common/libcommon.a(cmd_bootm.o)
                0x33f85070                print_image_hdr
                0x33f8504c                do_bootd
                0x33f857f4                gunzip
                0x33f85950                do_bootm
                0x33f85778                do_iminfo
 .text          0x33f86034      0x154 common/libcommon.a(cmd_cache.o)
                0x33f86078                do_dcache
                0x33f86100                do_icache
 .text          0x33f86188       0xd8 common/libcommon.a(cmd_console.o)
                0x33f86188                do_coninfo
 .text          0x33f86260      0x33c common/libcommon.a(cmd_date.o)
                0x33f86490                do_date
                0x33f862a8                mk_date
 .text          0x33f8659c      0x394 common/libcommon.a(cmd_elf.o)
                0x33f86888                do_bootelf
                0x33f8670c                do_bootvx
                0x33f8659c                valid_elf_image
                0x33f865f0                load_elf_image
 .text          0x33f86930      0xbd4 common/libcommon.a(cmd_flash.o)
                0x33f86e00                do_flinfo
                0x33f86e9c                flash_sect_erase
                0x33f87238                do_protect
                0x33f86f80                do_flerase
                0x33f87144                flash_sect_protect
 .text          0x33f87504      0x2f0 common/libcommon.a(cmd_itest.o)
                0x33f8756c                binary_test
                0x33f87748                do_itest
 .text          0x33f877f4      0xe4c common/libcommon.a(cmd_load.o)
                0x33f87cf0                k_data_init
                0x33f87b80                s1_sendpacket
                0x33f87e54                handle_send_packet
                0x33f87d7c                k_data_restore
                0x33f87c10                send_nack
                0x33f88088                do_load_serial_bin
                0x33f87de0                k_data_char
                0x33f87b50                chk1
                0x33f87d18                k_data_save
                0x33f87b24                ktrans
                0x33f87ae8                send_pad
                0x33f87bac                send_ack
                0x33f877f4                do_load_serial
 .text          0x33f88640      0xb20 common/libcommon.a(cmd_mem.o)
                0x33f88c7c                do_mem_base
                0x33f888c0                do_mem_mw
                0x33f890a8                do_mem_crc
                0x33f89058                do_mem_nm
                0x33f89080                do_mem_mm
                0x33f88b48                do_mem_cp
                0x33f88dc4                do_mem_mtest
                0x33f8898c                do_mem_cmp
                0x33f88640                cmd_get_data_size
                0x33f88cc0                do_mem_loop
                0x33f886b4                do_mem_md
 .text          0x33f89160       0x9c common/libcommon.a(cmd_misc.o)
                0x33f89160                do_sleep
 .text          0x33f891fc      0x2f0 common/libcommon.a(cmd_net.o)
                0x33f894c8                do_rarpb
                0x33f894d4                do_tftpb
                0x33f894e0                do_bootp
                0x33f894bc                do_nfs
 .text          0x33f894ec      0x898 common/libcommon.a(cmd_nvedit.o)
                0x33f89c18                getenv
                0x33f8971c                _do_setenv
                0x33f89c94                getenv_r
                0x33f89560                do_printenv
                0x33f89ba0                setenv
                0x33f89d58                do_saveenv
                0x33f89bd8                do_setenv
 .text          0x33f89d84      0x308 common/libcommon.a(command.o)
                0x33f89da4                do_echo
                0x33f89e24                find_cmd
                0x33f89ecc                do_help
                0x33f89d84                do_version
 .text          0x33f8a08c      0x570 common/libcommon.a(console.o)
                0x33f8a470                console_init_r
                0x33f8a2cc                printf
                0x33f8a3d0                console_assign
                0x33f8a258                getc
                0x33f8a2b0                puts
                0x33f8a3c4                dbg
                0x33f8a134                serial_printf
                0x33f8a194                ftstc
                0x33f8a218                fprintf
                0x33f8a270                tstc
                0x33f8a304                vprintf
                0x33f8a330                ctrlc
                0x33f8a288                putc
                0x33f8a388                disable_ctrlc
                0x33f8a16c                fgetc
                0x33f8a3a0                had_ctrlc
                0x33f8a1bc                fputc
                0x33f8a460                console_init_f
                0x33f8a3b0                clear_ctrlc
                0x33f8a1ec                fputs
 .text          0x33f8a5fc       0xf0 common/libcommon.a(devices.o)
                0x33f8a5fc                device_register
                0x33f8a6d0                devices_done
                0x33f8a620                devices_init
 .text          0x33f8a6ec     0x1088 common/libcommon.a(dlmalloc.o)
                0x33f8aa0c                malloc
                0x33f8b5d0                pvalloc
                0x33f8b5e8                calloc
                0x33f8b6bc                malloc_usable_size
                0x33f8b050                realloc
                0x33f8a720                malloc_trim
                0x33f8a6ec                malloc_bin_reloc
                0x33f8b6fc                mallopt
                0x33f8b4b4                memalign
                0x33f8b6b8                cfree
                0x33f8b5c4                valloc
                0x33f8a7f8                free
 .text          0x33f8b774      0x124 common/libcommon.a(env_common.o)
                0x33f8b7e8                env_get_addr
                0x33f8b808                env_relocate
                0x33f8b774                env_crc_update
                0x33f8b7c8                env_get_char_memory
 .text          0x33f8b898      0x144 common/libcommon.a(env_flash.o)
                0x33f8b9bc                env_relocate_spec
                0x33f8b8fc                saveenv
                0x33f8b898                env_get_char_spec
                0x33f8b8a4                env_init
 .text          0x33f8b9dc       0xc0 common/libcommon.a(exports.o)
                0x33f8b9e8                jumptable_init
                0x33f8b9e0                get_version
 .text          0x33f8ba9c      0x3c8 common/libcommon.a(flash.o)
                0x33f8bbec                flash_write
                0x33f8ba9c                flash_protect
                0x33f8bba4                addr2info
                0x33f8bd78                flash_perror
 .text          0x33f8be64      0x3c8 common/libcommon.a(lists.o)
                0x33f8bec4                DisposeHandle
                0x33f8bfd0                ListDispose
                0x33f8bfd4                ListInsertItems
                0x33f8bfbc                ListSetAllocationPolicy
                0x33f8c214                ListGetItemSize
                0x33f8c208                ListGetDataPtr
                0x33f8be64                NewHandle
                0x33f8beec                SetHandleSize
                0x33f8c188                ListInsertItem
                0x33f8bee4                GetHandleSize
                0x33f8c220                ListNumItems
                0x33f8c1d8                ListGetPtrToItem
                0x33f8bf5c                ListCreate
                0x33f8c190                ListGetItems
 .text          0x33f8c22c      0x2f8 common/libcommon.a(s_record.o)
                0x33f8c2a0                srec_decode
 .text          0x33f8c524      0xa98 common/libcommon.a(xyzModem.o)
                0x33f8cf20                xyzModem_error
                0x33f8cdf0                xyzModem_stream_close
                0x33f8c524                CYGACC_COMM_IF_GETC_TIMEOUT
                0x33f8c58c                parse_num
                0x33f8ce48                xyzModem_stream_terminate
                0x33f8c9d4                xyzModem_stream_open
                0x33f8c580                CYGACC_COMM_IF_PUTC
                0x33f8cb48                xyzModem_stream_read
 .text          0x33f8cfbc       0x40 common/libcommon.a(crc16.o)
                0x33f8cfbc                cyg_crc16
 .text          0x33f8cffc       0xfc lib_generic/libgeneric.a(crc32.o)
                0x33f8cffc                crc32
 .text          0x33f8d0f8       0xb4 lib_generic/libgeneric.a(display_options.o)
                0x33f8d0f8                display_options
                0x33f8d118                print_size
 .text          0x33f8d1ac      0x5a0 lib_generic/libgeneric.a(string.o)
                0x33f8d1ac                strcpy
                0x33f8d690                memscan
                0x33f8d5fc                memmove
                0x33f8d5d4                memcpy
                0x33f8d528                strswab
                0x33f8d35c                strnlen
                0x33f8d324                strrchr
                0x33f8d1ec                strcat
                0x33f8d71c                memchr
                0x33f8d6b4                strstr
                0x33f8d288                strncmp
                0x33f8d1c8                strncpy
                0x33f8d5a8                bcopy
                0x33f8d46c                strtok
                0x33f8d65c                memcmp
                0x33f8d218                strncat
                0x33f8d394                strdup
                0x33f8d584                memset
                0x33f8d258                strcmp
                0x33f8d4f0                strsep
                0x33f8d3cc                strspn
                0x33f8d300                strlen
                0x33f8d2d0                strchr
                0x33f8d42c                strpbrk
 .text          0x33f8d74c      0x7a8 lib_generic/libgeneric.a(vsprintf.o)
                0x33f8daa8                vsprintf
                0x33f8d804                simple_strtol
                0x33f8deac                panic
                0x33f8de8c                sprintf
                0x33f8d74c                simple_strtoul
 .text          0x33f8def4     0x2bd8 lib_generic/libgeneric.a(zlib.o)
                0x33f8ecc0                inflate
                0x33f8e238                inflateInit2
                0x33f8e3f0                inflateIncomp
                0x33f90958                adler32
                0x33f8e0c4                inflateReset
                0x33f8e12c                inflateSync
                0x33f8e398                inflateInit
                0x33f8e024                inflateEnd
 .text          0x33f90acc      0x114 board/ami/libami.a(ami.o)
                0x33f90bc0                dram_init
                0x33f90acc                board_init
 .text          0x33f90be0      0x704 board/ami/libami.a(flash.o)
                0x33f90be0                flash_identification
                0x33f90f4c                flash_erase
                0x33f90ccc                flash_init
                0x33f90e1c                flash_print_info
                0x33f91240                write_buff
 .text          0x33f912e4      0x118 cpu/arm920t/libarm920t.a(cpu.o)
                0x33f91324                cleanup_before_linux
                0x33f913b0                dcache_enable
                0x33f9131c                cpu_init
                0x33f91364                icache_enable
                0x33f9134c                do_reset
                0x33f91380                icache_disable
                0x33f913e8                dcache_status
                0x33f9139c                icache_status
                0x33f913cc                dcache_disable
 .text          0x33f913fc       0xdc cpu/arm920t/s3c24x0/libs3c24x0.a(serial.o)
                0x33f913fc                serial_setbrg
                0x33f914a0                serial_tstc
                0x33f91478                serial_putc
                0x33f91450                serial_init
                0x33f914b0                serial_puts
                0x33f91460                serial_getc
 *fill*         0x33f914d8        0x8 00
 .text          0x33f914e0      0x140 lib_arm/libarm.a(_divsi3.o)
                0x33f914e0                __divsi3
 .text          0x33f91620      0x100 lib_arm/libarm.a(_modsi3.o)
                0x33f91620                __modsi3
 .text          0x33f91720       0xb4 lib_arm/libarm.a(_umodsi3.o)
                0x33f91720                __umodsi3
 .text          0x33f917d4      0x274 lib_arm/libarm.a(armlinux.o)
                0x33f917d4                do_bootm_linux
 .text          0x33f91a48        0x4 lib_arm/libarm.a(cache.o)
                0x33f91a48                flush_cache
 .text          0x33f91a4c      0x2b8 rtc/librtc.a(date.o)
                0x33f91a4c                GregorianDay
                0x33f91c64                mktime
                0x33f91b3c                to_tm
 .text          0x33f91d04      0x214 rtc/librtc.a(s3c24x0_rtc.o)
                0x33f91e3c                rtc_set
                0x33f91ef4                rtc_reset
                0x33f91d50                rtc_get

.glue_7         0x33f91f18        0x0

.glue_7t        0x33f91f18        0x0
                0x33f91f18                . = ALIGN (0x4)

.rodata         0x33f91f18      0x6fc
 *(.rodata)
 .rodata        0x33f91f18       0x80 cpu/arm920t/libarm920t.a(interrupts.o)
 .rodata        0x33f91f98       0x28 lib_arm/libarm.a(board.o)
                0x33f91f98                version_string
 .rodata        0x33f91fc0        0x8 net/libnet.a(net.o)
 .rodata        0x33f91fc8        0x8 drivers/libdrivers.a(cs8900.o)
 .rodata        0x33f91fd0       0x14 common/libcommon.a(cmd_nvedit.o)
 .rodata        0x33f91fe4      0x200 common/libcommon.a(crc16.o)
 .rodata        0x33f921e4      0x400 lib_generic/libgeneric.a(crc32.o)
 .rodata        0x33f925e4       0x30 rtc/librtc.a(date.o)

.rodata.str1.4  0x33f92614     0x3c27
 .rodata.str1.4
                0x33f92614      0x293 cpu/arm920t/libarm920t.a(interrupts.o)
                                0x29c (size before relaxing)
 *fill*         0x33f928a7        0x1 00
 .rodata.str1.4
                0x33f928a8       0x75 lib_arm/libarm.a(board.o)
                                 0x7c (size before relaxing)
 *fill*         0x33f9291d        0x3 00
 .rodata.str1.4
                0x33f92920      0x1c9 net/libnet.a(net.o)
                                0x1cc (size before relaxing)
 *fill*         0x33f92ae9        0x3 00
 .rodata.str1.4
                0x33f92aec      0x1cb net/libnet.a(tftp.o)
                                0x1d4 (size before relaxing)
 *fill*         0x33f92cb7        0x1 00
 .rodata.str1.4
                0x33f92cb8       0x84 net/libnet.a(bootp.o)
                                 0xb8 (size before relaxing)
 .rodata.str1.4
                0x33f92d3c       0x13 net/libnet.a(rarp.o)
                                 0x4c (size before relaxing)
 *fill*         0x33f92d4f        0x1 00
 .rodata.str1.4
                0x33f92d50      0x101 net/libnet.a(nfs.o)
                                0x18c (size before relaxing)
 *fill*         0x33f92e51        0x3 00
 .rodata.str1.4
                0x33f92e54       0xd2 drivers/libdrivers.a(cs8900.o)
                                 0xdc (size before relaxing)
 *fill*         0x33f92f26        0x2 00
 .rodata.str1.4
                0x33f92f28       0xfc common/libcommon.a(main.o)
 .rodata.str1.4
                0x33f93024       0xf6 common/libcommon.a(cmd_autoscript.o)
                                 0xf8 (size before relaxing)
 *fill*         0x33f9311a        0x2 00
 .rodata.str1.4
                0x33f9311c       0xbf common/libcommon.a(cmd_bdinfo.o)
                                 0xc0 (size before relaxing)
 *fill*         0x33f931db        0x1 00
 .rodata.str1.4
                0x33f931dc      0x10b common/libcommon.a(cmd_boot.o)
                                0x118 (size before relaxing)
 *fill*         0x33f932e7        0x1 00
 .rodata.str1.4
                0x33f932e8      0x8b1 common/libcommon.a(cmd_bootm.o)
                                0x8f4 (size before relaxing)
 *fill*         0x33f93b99        0x3 00
 .rodata.str1.4
                0x33f93b9c      0x125 common/libcommon.a(cmd_cache.o)
                                0x13c (size before relaxing)
 *fill*         0x33f93cc1        0x3 00
 .rodata.str1.4
                0x33f93cc4       0x70 common/libcommon.a(cmd_console.o)
                                 0x74 (size before relaxing)
 .rodata.str1.4
                0x33f93d34      0x16c common/libcommon.a(cmd_date.o)
                                0x180 (size before relaxing)
 .rodata.str1.4
                0x33f93ea0      0x2d7 common/libcommon.a(cmd_elf.o)
                                0x2f0 (size before relaxing)
 *fill*         0x33f94177        0x1 00
 .rodata.str1.4
                0x33f94178      0x767 common/libcommon.a(cmd_flash.o)
                                0x780 (size before relaxing)
 *fill*         0x33f948df        0x1 00
 .rodata.str1.4
                0x33f948e0       0xce common/libcommon.a(cmd_itest.o)
                                 0xdc (size before relaxing)
 *fill*         0x33f949ae        0x2 00
 .rodata.str1.4
                0x33f949b0      0x37c common/libcommon.a(cmd_load.o)
                                0x398 (size before relaxing)
 .rodata.str1.4
                0x33f94d2c      0x629 common/libcommon.a(cmd_mem.o)
                                0x648 (size before relaxing)
 *fill*         0x33f95355        0x3 00
 .rodata.str1.4
                0x33f95358       0x70 common/libcommon.a(cmd_misc.o)
                                 0x7c (size before relaxing)
 .rodata.str1.4
                0x33f953c8      0x1ad common/libcommon.a(cmd_net.o)
                                0x1fc (size before relaxing)
 *fill*         0x33f95575        0x3 00
 .rodata.str1.4
                0x33f95578      0x2e5 common/libcommon.a(cmd_nvedit.o)
                                0x378 (size before relaxing)
 *fill*         0x33f9585d        0x3 00
 .rodata.str1.4
                0x33f95860      0x27e common/libcommon.a(command.o)
                                0x280 (size before relaxing)
 *fill*         0x33f95ade        0x2 00
 .rodata.str1.4
                0x33f95ae0       0x75 common/libcommon.a(console.o)
                                 0x7c (size before relaxing)
 *fill*         0x33f95b55        0x3 00
 .rodata.str1.4
                0x33f95b58       0x2f common/libcommon.a(devices.o)
                                 0x48 (size before relaxing)
 *fill*         0x33f95b87        0x1 00
 .rodata.str1.4
                0x33f95b88       0x33 common/libcommon.a(env_common.o)
                                 0x34 (size before relaxing)
 *fill*         0x33f95bbb        0x1 00
 .rodata.str1.4
                0x33f95bbc       0x31 common/libcommon.a(env_flash.o)
                                 0x3c (size before relaxing)
 *fill*         0x33f95bed        0x3 00
 .rodata.str1.4
                0x33f95bf0      0x11d common/libcommon.a(flash.o)
                                0x120 (size before relaxing)
 *fill*         0x33f95d0d        0x3 00
 .rodata.str1.4
                0x33f95d10       0xf2 common/libcommon.a(xyzModem.o)
                                 0xf8 (size before relaxing)
 *fill*         0x33f95e02        0x2 00
 .rodata.str1.4
                0x33f95e04       0x17 lib_generic/libgeneric.a(display_options.o)
                                 0x20 (size before relaxing)
 *fill*         0x33f95e1b        0x1 00
 .rodata.str1.4
                0x33f95e1c       0x57 lib_generic/libgeneric.a(vsprintf.o)
                                 0x58 (size before relaxing)
 *fill*         0x33f95e73        0x1 00
 .rodata.str1.4
                0x33f95e74      0x20d lib_generic/libgeneric.a(zlib.o)
                                0x214 (size before relaxing)
 *fill*         0x33f96081        0x3 00
 .rodata.str1.4
                0x33f96084      0x15c board/ami/libami.a(flash.o)
                                0x160 (size before relaxing)
 .rodata.str1.4
                0x33f961e0       0x5b lib_arm/libarm.a(armlinux.o)
                                 0xb8 (size before relaxing)
                0x33f9623c                . = ALIGN (0x4)

.data           0x33f9623c      0x96c
 *(.data)
 .data          0x33f9623c       0x2c lib_arm/libarm.a(board.o)
                0x33f9623c                init_sequence
 .data          0x33f96268        0xa net/libnet.a(net.o)
                0x33f9626c                NetBcastAddr
                0x33f96268                NetOurNativeVLAN
                0x33f9626a                NetOurVLAN
 *fill*         0x33f96272        0x2 00
 .data          0x33f96274        0x4 net/libnet.a(nfs.o)
 .data          0x33f96278       0x10 common/libcommon.a(main.o)
 .data          0x33f96288        0x4 common/libcommon.a(cmd_bootm.o)
                0x33f96288                load_addr
 .data          0x33f9628c       0x1c common/libcommon.a(cmd_date.o)
                0x33f9628c                weekdays
 .data          0x33f962a8       0x68 common/libcommon.a(cmd_itest.o)
                0x33f962a8                op_table
 .data          0x33f96310        0x4 common/libcommon.a(cmd_load.o)
 .data          0x33f96314        0x4 common/libcommon.a(cmd_mem.o)
                0x33f96314                dp_last_length
 .data          0x33f96318        0xc common/libcommon.a(devices.o)
                0x33f96318                stdio_names
 .data          0x33f96324      0x414 common/libcommon.a(dlmalloc.o)
 .data          0x33f96738       0x5c common/libcommon.a(env_common.o)
                0x33f96790                env_get_char
                0x33f96738                default_environment
 .data          0x33f96794        0xc common/libcommon.a(env_flash.o)
                0x33f96798                env_name_spec
                0x33f96794                env_ptr
 .data          0x33f967a0      0x2a0 lib_generic/libgeneric.a(zlib.o)
                0x33f967c0                zlib_version
                0x33f967a0                z_errmsg
 .data          0x33f96a40      0x100 lib_generic/libgeneric.a(ctype.o)
                0x33f96a40                _ctype
 .data          0x33f96b40       0x38 board/ami/libami.a(flash.o)
                0x33f96b60                OrgAT49BV16x4
                0x33f96b40                OrgAT49BV322A
                0x33f96b50                OrgAT49BV16x4A
 .data          0x33f96b78       0x30 rtc/librtc.a(date.o)
                0x33f96ba8                . = ALIGN (0x4)

.got
 *(.got)
                0x33f96ba8                . = .
                0x33f96ba8                __u_boot_cmd_start = .

.u_boot_cmd     0x33f96ba8      0x438
 *(.u_boot_cmd)
 .u_boot_cmd    0x33f96ba8       0x18 common/libcommon.a(cmd_autoscript.o)
                0x33f96ba8                __u_boot_cmd_autoscr
 .u_boot_cmd    0x33f96bc0       0x18 common/libcommon.a(cmd_bdinfo.o)
                0x33f96bc0                __u_boot_cmd_bdinfo
 .u_boot_cmd    0x33f96bd8       0x30 common/libcommon.a(cmd_boot.o)
                0x33f96bd8                __u_boot_cmd_reset
                0x33f96bf0                __u_boot_cmd_go
 .u_boot_cmd    0x33f96c08       0x78 common/libcommon.a(cmd_bootm.o)
                0x33f96c68                __u_boot_cmd_bootm
                0x33f96c20                __u_boot_cmd_iminfo
                0x33f96c38                __u_boot_cmd_bootd
                0x33f96c50                __u_boot_cmd_boot
                0x33f96c08                __u_boot_cmd_imls
 .u_boot_cmd    0x33f96c80       0x30 common/libcommon.a(cmd_cache.o)
                0x33f96c80                __u_boot_cmd_dcache
                0x33f96c98                __u_boot_cmd_icache
 .u_boot_cmd    0x33f96cb0       0x18 common/libcommon.a(cmd_console.o)
                0x33f96cb0                __u_boot_cmd_coninfo
 .u_boot_cmd    0x33f96cc8       0x18 common/libcommon.a(cmd_date.o)
                0x33f96cc8                __u_boot_cmd_date
 .u_boot_cmd    0x33f96ce0       0x30 common/libcommon.a(cmd_elf.o)
                0x33f96ce0                __u_boot_cmd_bootvx
                0x33f96cf8                __u_boot_cmd_bootelf
 .u_boot_cmd    0x33f96d10       0x48 common/libcommon.a(cmd_flash.o)
                0x33f96d40                __u_boot_cmd_flinfo
                0x33f96d28                __u_boot_cmd_erase
                0x33f96d10                __u_boot_cmd_protect
 .u_boot_cmd    0x33f96d58       0x18 common/libcommon.a(cmd_itest.o)
                0x33f96d58                __u_boot_cmd_itest
 .u_boot_cmd    0x33f96d70       0x48 common/libcommon.a(cmd_load.o)
                0x33f96d70                __u_boot_cmd_loady
                0x33f96d88                __u_boot_cmd_loadb
                0x33f96da0                __u_boot_cmd_loads
 .u_boot_cmd    0x33f96db8       0xf0 common/libcommon.a(cmd_mem.o)
                0x33f96e90                __u_boot_cmd_md
                0x33f96e18                __u_boot_cmd_cmp
                0x33f96e48                __u_boot_cmd_mw
                0x33f96dd0                __u_boot_cmd_loop
                0x33f96de8                __u_boot_cmd_base
                0x33f96e78                __u_boot_cmd_mm
                0x33f96e00                __u_boot_cmd_crc32
                0x33f96e60                __u_boot_cmd_nm
                0x33f96db8                __u_boot_cmd_mtest
                0x33f96e30                __u_boot_cmd_cp
 .u_boot_cmd    0x33f96ea8       0x18 common/libcommon.a(cmd_misc.o)
                0x33f96ea8                __u_boot_cmd_sleep
 .u_boot_cmd    0x33f96ec0       0x60 common/libcommon.a(cmd_net.o)
                0x33f96ec0                __u_boot_cmd_nfs
                0x33f96ed8                __u_boot_cmd_rarpboot
                0x33f96ef0                __u_boot_cmd_tftpboot
                0x33f96f08                __u_boot_cmd_bootp
 .u_boot_cmd    0x33f96f20       0x60 common/libcommon.a(cmd_nvedit.o)
                0x33f96f20                __u_boot_cmd_run
                0x33f96f38                __u_boot_cmd_saveenv
                0x33f96f68                __u_boot_cmd_printenv
                0x33f96f50                __u_boot_cmd_setenv
 .u_boot_cmd    0x33f96f80       0x60 common/libcommon.a(command.o)
                0x33f96fb0                __u_boot_cmd_echo
                0x33f96f80                __u_boot_cmd_question_mark
                0x33f96fc8                __u_boot_cmd_version
                0x33f96f98                __u_boot_cmd_help
                0x33f96fe0                __u_boot_cmd_end = .
                0x33f96fe0                . = ALIGN (0x4)
                0x33f96fe0                __bss_start = .

.bss            0x33f96fe0     0x4854
 *(.bss)
 .bss           0x33f96fe0        0xc cpu/arm920t/s3c24x0/libs3c24x0.a(interrupts.o)
                0x33f96fe0                timer_load_val
 .bss           0x33f96fec       0x10 lib_arm/libarm.a(board.o)
                0x33f96fec                monitor_flash_len
 .bss           0x33f96ffc     0x25c0 net/libnet.a(net.o)
                0x33f995a8                NetArpWaitTry
                0x33f98f78                NetArpWaitPacketMAC
                0x33f970a0                NetOurEther
                0x33f970a8                NetOurIP
                0x33f970ac                NetServerIP
                0x33f98f80                NetArpWaitTxPacketSize
                0x33f98f74                NetArpWaitReplyIP
                0x33f970b0                NetRxPackets
                0x33f98f7c                NetArpWaitTxPacket
                0x33f9706e                NetOurNISDomain
                0x33f98f70                NetArpWaitPacketIP
                0x33f970cc                NetState
                0x33f970d0                BootFile
                0x33f97006                NetServerEther
                0x33f97098                NetOurSubnetMask
                0x33f9700c                NetBootFileSize
                0x33f970c8                NetIPID
                0x33f9704e                NetOurHostName
                0x33f970c0                NetRxPkt
                0x33f97094                NetOurGatewayIP
                0x33f97000                NetEtherNullAddr
                0x33f98f84                NetArpWaitPacketBuf
                0x33f970c4                NetRxPktLen
                0x33f96ffc                NetTxPacket
                0x33f9709c                NetBootFileXferSize
                0x33f97090                NetOurDNSIP
                0x33f97150                PktBuf
                0x33f9700e                NetOurRootPath
                0x33f995a4                NetArpWaitTimerStart
 .bss           0x33f995bc       0x34 net/libnet.a(tftp.o)
 .bss           0x33f995f0        0x8 net/libnet.a(bootp.o)
                0x33f995f4                BootpTry
                0x33f995f0                BootpID
 .bss           0x33f995f8        0x4 net/libnet.a(rarp.o)
                0x33f995f8                RarpTry
 .bss           0x33f995fc      0x8b0 net/libnet.a(nfs.o)
 .bss           0x33f99eac      0x200 common/libcommon.a(main.o)
                0x33f99eac                console_buffer
 .bss           0x33f9a0ac       0x40 common/libcommon.a(cmd_bootm.o)
                0x33f9a0ac                header
 .bss           0x33f9a0ec       0x88 common/libcommon.a(cmd_load.o)
                0x33f9a118                his_pad_char
                0x33f9a0ec                os_data_count
                0x33f9a11c                os_data_init
                0x33f9a138                send_ptr
                0x33f9a0f0                os_data_header
                0x33f9a120                os_data_char
                0x33f9a110                his_eol
                0x33f9a119                his_quote
                0x33f9a124                send_parms
                0x33f9a114                his_pad_count
 .bss           0x33f9a174       0x14 common/libcommon.a(cmd_mem.o)
                0x33f9a178                dp_last_size
                0x33f9a174                dp_last_addr
                0x33f9a180                mm_last_size
                0x33f9a17c                mm_last_addr
 .bss           0x33f9a188        0x8 common/libcommon.a(console.o)
 .bss           0x33f9a190       0x10 common/libcommon.a(devices.o)
                0x33f9a19c                devlist
                0x33f9a190                stdio_devices
 .bss           0x33f9a1a0       0x3c common/libcommon.a(dlmalloc.o)
 .bss           0x33f9a1dc      0x43c common/libcommon.a(xyzModem.o)
 .bss           0x33f9a618        0x4 lib_generic/libgeneric.a(string.o)
                0x33f9a618                ___strtok
 .bss           0x33f9a61c     0x10a8 lib_generic/libgeneric.a(zlib.o)
 .bss           0x33f9b6c4      0x170 board/ami/libami.a(flash.o)
                0x33f9b6c4                flash_info
                0x33f9b834                _end = .
Address of section .text set to 0x33f80000
LOAD cpu/arm920t/start.o
START GROUP
LOAD lib_generic/libgeneric.a
LOAD board/ami/libami.a
LOAD cpu/arm920t/libarm920t.a
LOAD cpu/arm920t/s3c24x0/libs3c24x0.a
LOAD lib_arm/libarm.a
LOAD fs/cramfs/libcramfs.a
LOAD fs/fat/libfat.a
LOAD fs/fdos/libfdos.a
LOAD fs/jffs2/libjffs2.a
LOAD fs/reiserfs/libreiserfs.a
LOAD fs/ext2/libext2fs.a
LOAD net/libnet.a
LOAD disk/libdisk.a
LOAD rtc/librtc.a
LOAD dtt/libdtt.a
LOAD drivers/libdrivers.a
LOAD drivers/nand/libnand.a
LOAD drivers/nand_legacy/libnand_legacy.a
LOAD drivers/sk98lin/libsk98lin.a
LOAD post/libpost.a
LOAD post/cpu/libcpu.a
LOAD common/libcommon.a
END GROUP
LOAD /work/toolchains/armtools/bin/../lib/gcc/arm-linux/3.4.2/libgcc.a
OUTPUT(u-boot elf32-littlearm)

.stab           0x00000000      0xbc4
 .stab          0x00000000      0x408 cpu/arm920t/start.o
 .stab          0x00000408       0x90 board/ami/libami.a(lowlevel_init.o)
                                 0x9c (size before relaxing)
 .stab          0x00000498      0x210 lib_arm/libarm.a(_udivsi3.o)
                                0x21c (size before relaxing)
 .stab          0x000006a8      0x1b0 lib_arm/libarm.a(_divsi3.o)
                                0x1bc (size before relaxing)
 .stab          0x00000858      0x108 lib_arm/libarm.a(_modsi3.o)
                                0x114 (size before relaxing)
 .stab          0x00000960      0x264 lib_arm/libarm.a(_umodsi3.o)
                                0x270 (size before relaxing)

.stabstr        0x00000000       0x54
 .stabstr       0x00000000       0x54 cpu/arm920t/start.o
                                  0x0 (size before relaxing)

.debug_abbrev   0x00000000     0x4e2a
 .debug_abbrev  0x00000000       0xe0 cpu/arm920t/libarm920t.a(interrupts.o)
 .debug_abbrev  0x000000e0      0x1c8 cpu/arm920t/s3c24x0/libs3c24x0.a(interrupts.o)
 .debug_abbrev  0x000002a8       0xf8 cpu/arm920t/s3c24x0/libs3c24x0.a(speed.o)
 .debug_abbrev  0x000003a0      0x1fc lib_arm/libarm.a(board.o)
 .debug_abbrev  0x0000059c       0x3a lib_arm/libarm.a(div0.o)
 .debug_abbrev  0x000005d6      0x2e2 net/libnet.a(net.o)
 .debug_abbrev  0x000008b8      0x19e net/libnet.a(tftp.o)
 .debug_abbrev  0x00000a56      0x261 net/libnet.a(bootp.o)
 .debug_abbrev  0x00000cb7      0x108 net/libnet.a(rarp.o)
 .debug_abbrev  0x00000dbf       0xac net/libnet.a(eth.o)
 .debug_abbrev  0x00000e6b      0x2e3 net/libnet.a(nfs.o)
 .debug_abbrev  0x0000114e      0x1d7 drivers/libdrivers.a(cs8900.o)
 .debug_abbrev  0x00001325      0x1fb common/libcommon.a(main.o)
 .debug_abbrev  0x00001520      0x141 common/libcommon.a(cmd_autoscript.o)
 .debug_abbrev  0x00001661      0x119 common/libcommon.a(cmd_bdinfo.o)
 .debug_abbrev  0x0000177a       0xd6 common/libcommon.a(cmd_boot.o)
 .debug_abbrev  0x00001850      0x2cf common/libcommon.a(cmd_bootm.o)
 .debug_abbrev  0x00001b1f       0xe5 common/libcommon.a(cmd_cache.o)
 .debug_abbrev  0x00001c04      0x134 common/libcommon.a(cmd_console.o)
 .debug_abbrev  0x00001d38      0x15a common/libcommon.a(cmd_date.o)
 .debug_abbrev  0x00001e92      0x178 common/libcommon.a(cmd_elf.o)
 .debug_abbrev  0x0000200a      0x1a4 common/libcommon.a(cmd_flash.o)
 .debug_abbrev  0x000021ae      0x17f common/libcommon.a(cmd_itest.o)
 .debug_abbrev  0x0000232d      0x301 common/libcommon.a(cmd_load.o)
 .debug_abbrev  0x0000262e      0x1c0 common/libcommon.a(cmd_mem.o)
 .debug_abbrev  0x000027ee       0xc7 common/libcommon.a(cmd_misc.o)
 .debug_abbrev  0x000028b5      0x17b common/libcommon.a(cmd_net.o)
 .debug_abbrev  0x00002a30      0x22e common/libcommon.a(cmd_nvedit.o)
 .debug_abbrev  0x00002c5e      0x18b common/libcommon.a(command.o)
 .debug_abbrev  0x00002de9      0x23a common/libcommon.a(console.o)
 .debug_abbrev  0x00003023      0x15b common/libcommon.a(devices.o)
 .debug_abbrev  0x0000317e      0x1d6 common/libcommon.a(dlmalloc.o)
 .debug_abbrev  0x00003354      0x149 common/libcommon.a(env_common.o)
 .debug_abbrev  0x0000349d      0x180 common/libcommon.a(env_flash.o)
 .debug_abbrev  0x0000361d       0xf3 common/libcommon.a(exports.o)
 .debug_abbrev  0x00003710      0x116 common/libcommon.a(flash.o)
 .debug_abbrev  0x00003826      0x18e common/libcommon.a(lists.o)
 .debug_abbrev  0x000039b4       0xac common/libcommon.a(s_record.o)
 .debug_abbrev  0x00003a60      0x214 common/libcommon.a(xyzModem.o)
 .debug_abbrev  0x00003c74       0x9f common/libcommon.a(crc16.o)
 .debug_abbrev  0x00003d13       0x90 lib_generic/libgeneric.a(crc32.o)
 .debug_abbrev  0x00003da3       0xc3 lib_generic/libgeneric.a(display_options.o)
 .debug_abbrev  0x00003e66      0x136 lib_generic/libgeneric.a(string.o)
 .debug_abbrev  0x00003f9c      0x1ad lib_generic/libgeneric.a(vsprintf.o)
 .debug_abbrev  0x00004149      0x271 lib_generic/libgeneric.a(zlib.o)
 .debug_abbrev  0x000043ba       0x42 lib_generic/libgeneric.a(ctype.o)
 .debug_abbrev  0x000043fc      0x17a board/ami/libami.a(ami.o)
 .debug_abbrev  0x00004576      0x1b7 board/ami/libami.a(flash.o)
 .debug_abbrev  0x0000472d      0x124 cpu/arm920t/libarm920t.a(cpu.o)
 .debug_abbrev  0x00004851      0x17c cpu/arm920t/s3c24x0/libs3c24x0.a(serial.o)
 .debug_abbrev  0x000049cd      0x173 lib_arm/libarm.a(armlinux.o)
 .debug_abbrev  0x00004b40       0x4e lib_arm/libarm.a(cache.o)
 .debug_abbrev  0x00004b8e       0xdc rtc/librtc.a(date.o)
 .debug_abbrev  0x00004c6a      0x1c0 rtc/librtc.a(s3c24x0_rtc.o)

.debug_info     0x00000000    0x12728
 .debug_info    0x00000000      0x242 cpu/arm920t/libarm920t.a(interrupts.o)
 .debug_info    0x00000242      0x439 cpu/arm920t/s3c24x0/libs3c24x0.a(interrupts.o)
 .debug_info    0x0000067b      0x1f2 cpu/arm920t/s3c24x0/libs3c24x0.a(speed.o)
 .debug_info    0x0000086d      0x4dd lib_arm/libarm.a(board.o)
 .debug_info    0x00000d4a       0x44 lib_arm/libarm.a(div0.o)
 .debug_info    0x00000d8e     0x14ed net/libnet.a(net.o)
 .debug_info    0x0000227b      0x41a net/libnet.a(tftp.o)
 .debug_info    0x00002695      0x8be net/libnet.a(bootp.o)
 .debug_info    0x00002f53      0x245 net/libnet.a(rarp.o)
 .debug_info    0x00003198      0x17d net/libnet.a(eth.o)
 .debug_info    0x00003315      0xe3a net/libnet.a(nfs.o)
 .debug_info    0x0000414f      0x489 drivers/libdrivers.a(cs8900.o)
 .debug_info    0x000045d8      0x621 common/libcommon.a(main.o)
 .debug_info    0x00004bf9      0x3fc common/libcommon.a(cmd_autoscript.o)
 .debug_info    0x00004ff5      0x368 common/libcommon.a(cmd_bdinfo.o)
 .debug_info    0x0000535d      0x1c8 common/libcommon.a(cmd_boot.o)
 .debug_info    0x00005525     0x1364 common/libcommon.a(cmd_bootm.o)
 .debug_info    0x00006889      0x218 common/libcommon.a(cmd_cache.o)
 .debug_info    0x00006aa1      0x37d common/libcommon.a(cmd_console.o)
 .debug_info    0x00006e1e      0x4fb common/libcommon.a(cmd_date.o)
 .debug_info    0x00007319      0x506 common/libcommon.a(cmd_elf.o)
 .debug_info    0x0000781f      0x7ae common/libcommon.a(cmd_flash.o)
 .debug_info    0x00007fcd      0x42a common/libcommon.a(cmd_itest.o)
 .debug_info    0x000083f7      0xd34 common/libcommon.a(cmd_load.o)
 .debug_info    0x0000912b      0xa16 common/libcommon.a(cmd_mem.o)
 .debug_info    0x00009b41      0x1aa common/libcommon.a(cmd_misc.o)
 .debug_info    0x00009ceb      0x4c3 common/libcommon.a(cmd_net.o)
 .debug_info    0x0000a1ae      0x825 common/libcommon.a(cmd_nvedit.o)
 .debug_info    0x0000a9d3      0x3f4 common/libcommon.a(command.o)
 .debug_info    0x0000adc7      0x855 common/libcommon.a(console.o)
 .debug_info    0x0000b61c      0x485 common/libcommon.a(devices.o)
 .debug_info    0x0000baa1      0xb59 common/libcommon.a(dlmalloc.o)
 .debug_info    0x0000c5fa      0x364 common/libcommon.a(env_common.o)
 .debug_info    0x0000c95e      0x376 common/libcommon.a(env_flash.o)
 .debug_info    0x0000ccd4      0x255 common/libcommon.a(exports.o)
 .debug_info    0x0000cf29      0x2f6 common/libcommon.a(flash.o)
 .debug_info    0x0000d21f      0x4df common/libcommon.a(lists.o)
 .debug_info    0x0000d6fe      0x17a common/libcommon.a(s_record.o)
 .debug_info    0x0000d878      0x625 common/libcommon.a(xyzModem.o)
 .debug_info    0x0000de9d      0x10f common/libcommon.a(crc16.o)
 .debug_info    0x0000dfac      0x12a lib_generic/libgeneric.a(crc32.o)
 .debug_info    0x0000e0d6      0x120 lib_generic/libgeneric.a(display_options.o)
 .debug_info    0x0000e1f6      0x828 lib_generic/libgeneric.a(string.o)
 .debug_info    0x0000ea1e      0x401 lib_generic/libgeneric.a(vsprintf.o)
 .debug_info    0x0000ee1f     0x16ca lib_generic/libgeneric.a(zlib.o)
 .debug_info    0x000104e9       0x56 lib_generic/libgeneric.a(ctype.o)
 .debug_info    0x0001053f      0x64c board/ami/libami.a(ami.o)
 .debug_info    0x00010b8b      0x4fc board/ami/libami.a(flash.o)
 .debug_info    0x00011087      0x2f0 cpu/arm920t/libarm920t.a(cpu.o)
 .debug_info    0x00011377      0x47f cpu/arm920t/s3c24x0/libs3c24x0.a(serial.o)
 .debug_info    0x000117f6      0x58b lib_arm/libarm.a(armlinux.o)
 .debug_info    0x00011d81       0xa8 lib_arm/libarm.a(cache.o)
 .debug_info    0x00011e29      0x253 rtc/librtc.a(date.o)
 .debug_info    0x0001207c      0x6ac rtc/librtc.a(s3c24x0_rtc.o)

.debug_line     0x00000000     0x53e0
 .debug_line    0x00000000       0xad cpu/arm920t/libarm920t.a(interrupts.o)
 .debug_line    0x000000ad      0x126 cpu/arm920t/s3c24x0/libs3c24x0.a(interrupts.o)
 .debug_line    0x000001d3       0xc6 cpu/arm920t/s3c24x0/libs3c24x0.a(speed.o)
 .debug_line    0x00000299      0x179 lib_arm/libarm.a(board.o)
 .debug_line    0x00000412       0x33 lib_arm/libarm.a(div0.o)
 .debug_line    0x00000445      0x5cf net/libnet.a(net.o)
 .debug_line    0x00000a14      0x23e net/libnet.a(tftp.o)
 .debug_line    0x00000c52      0x283 net/libnet.a(bootp.o)
 .debug_line    0x00000ed5       0xd4 net/libnet.a(rarp.o)
 .debug_line    0x00000fa9       0x95 net/libnet.a(eth.o)
 .debug_line    0x0000103e      0x45a net/libnet.a(nfs.o)
 .debug_line    0x00001498      0x15b drivers/libdrivers.a(cs8900.o)
 .debug_line    0x000015f3      0x1de common/libcommon.a(main.o)
 .debug_line    0x000017d1      0x1b6 common/libcommon.a(cmd_autoscript.o)
 .debug_line    0x00001987       0xef common/libcommon.a(cmd_bdinfo.o)
 .debug_line    0x00001a76       0xaf common/libcommon.a(cmd_boot.o)
 .debug_line    0x00001b25      0x4b4 common/libcommon.a(cmd_bootm.o)
 .debug_line    0x00001fd9       0x99 common/libcommon.a(cmd_cache.o)
 .debug_line    0x00002072       0x94 common/libcommon.a(cmd_console.o)
 .debug_line    0x00002106      0x130 common/libcommon.a(cmd_date.o)
 .debug_line    0x00002236      0x178 common/libcommon.a(cmd_elf.o)
 .debug_line    0x000023ae      0x224 common/libcommon.a(cmd_flash.o)
 .debug_line    0x000025d2       0xf4 common/libcommon.a(cmd_itest.o)
 .debug_line    0x000026c6      0x366 common/libcommon.a(cmd_load.o)
 .debug_line    0x00002a2c      0x273 common/libcommon.a(cmd_mem.o)
 .debug_line    0x00002c9f       0xa8 common/libcommon.a(cmd_misc.o)
 .debug_line    0x00002d47       0xfe common/libcommon.a(cmd_net.o)
 .debug_line    0x00002e45      0x263 common/libcommon.a(cmd_nvedit.o)
 .debug_line    0x000030a8       0xfe common/libcommon.a(command.o)
 .debug_line    0x000031a6      0x21b common/libcommon.a(console.o)
 .debug_line    0x000033c1      0x114 common/libcommon.a(devices.o)
 .debug_line    0x000034d5      0x369 common/libcommon.a(dlmalloc.o)
 .debug_line    0x0000383e      0x113 common/libcommon.a(env_common.o)
 .debug_line    0x00003951      0x129 common/libcommon.a(env_flash.o)
 .debug_line    0x00003a7a       0xb5 common/libcommon.a(exports.o)
 .debug_line    0x00003b2f      0x11f common/libcommon.a(flash.o)
 .debug_line    0x00003c4e       0xf2 common/libcommon.a(lists.o)
 .debug_line    0x00003d40       0xf4 common/libcommon.a(s_record.o)
 .debug_line    0x00003e34      0x215 common/libcommon.a(xyzModem.o)
 .debug_line    0x00004049       0x9a common/libcommon.a(crc16.o)
 .debug_line    0x000040e3       0x72 lib_generic/libgeneric.a(crc32.o)
 .debug_line    0x00004155       0x8c lib_generic/libgeneric.a(display_options.o)
 .debug_line    0x000041e1      0x194 lib_generic/libgeneric.a(string.o)
 .debug_line    0x00004375      0x1bd lib_generic/libgeneric.a(vsprintf.o)
 .debug_line    0x00004532      0x5bb lib_generic/libgeneric.a(zlib.o)
 .debug_line    0x00004aed       0x25 lib_generic/libgeneric.a(ctype.o)
 .debug_line    0x00004b12      0x122 board/ami/libami.a(ami.o)
 .debug_line    0x00004c34      0x1fe board/ami/libami.a(flash.o)
 .debug_line    0x00004e32       0xbd cpu/arm920t/libarm920t.a(cpu.o)
 .debug_line    0x00004eef      0x122 cpu/arm920t/s3c24x0/libs3c24x0.a(serial.o)
 .debug_line    0x00005011      0x1c8 lib_arm/libarm.a(armlinux.o)
 .debug_line    0x000051d9       0x34 lib_arm/libarm.a(cache.o)
 .debug_line    0x0000520d       0xb1 rtc/librtc.a(date.o)
 .debug_line    0x000052be      0x122 rtc/librtc.a(s3c24x0_rtc.o)

.debug_frame    0x00000000     0x263c
 .debug_frame   0x00000000      0x110 cpu/arm920t/libarm920t.a(interrupts.o)
 .debug_frame   0x00000110       0xf8 cpu/arm920t/s3c24x0/libs3c24x0.a(interrupts.o)
 .debug_frame   0x00000208       0x78 cpu/arm920t/s3c24x0/libs3c24x0.a(speed.o)
 .debug_frame   0x00000280       0x9c lib_arm/libarm.a(board.o)
 .debug_frame   0x0000031c       0x20 lib_arm/libarm.a(div0.o)
 .debug_frame   0x0000033c      0x270 net/libnet.a(net.o)
 .debug_frame   0x000005ac       0x8c net/libnet.a(tftp.o)
 .debug_frame   0x00000638       0x8c net/libnet.a(bootp.o)
 .debug_frame   0x000006c4       0x60 net/libnet.a(rarp.o)
 .debug_frame   0x00000724       0x20 net/libnet.a(eth.o)
 .debug_frame   0x00000744      0x150 net/libnet.a(nfs.o)
 .debug_frame   0x00000894      0x148 drivers/libdrivers.a(cs8900.o)
 .debug_frame   0x000009dc       0xb8 common/libcommon.a(main.o)
 .debug_frame   0x00000a94       0x4c common/libcommon.a(cmd_autoscript.o)
 .debug_frame   0x00000ae0       0x3c common/libcommon.a(cmd_bdinfo.o)
 .debug_frame   0x00000b1c       0x2c common/libcommon.a(cmd_boot.o)
 .debug_frame   0x00000b48      0x120 common/libcommon.a(cmd_bootm.o)
 .debug_frame   0x00000c68       0x58 common/libcommon.a(cmd_cache.o)
 .debug_frame   0x00000cc0       0x30 common/libcommon.a(cmd_console.o)
 .debug_frame   0x00000cf0       0x64 common/libcommon.a(cmd_date.o)
 .debug_frame   0x00000d54       0x88 common/libcommon.a(cmd_elf.o)
 .debug_frame   0x00000ddc      0x124 common/libcommon.a(cmd_flash.o)
 .debug_frame   0x00000f00       0x74 common/libcommon.a(cmd_itest.o)
 .debug_frame   0x00000f74      0x198 common/libcommon.a(cmd_load.o)
 .debug_frame   0x0000110c      0x184 common/libcommon.a(cmd_mem.o)
 .debug_frame   0x00001290       0x30 common/libcommon.a(cmd_misc.o)
 .debug_frame   0x000012c0       0x74 common/libcommon.a(cmd_net.o)
 .debug_frame   0x00001334      0x108 common/libcommon.a(cmd_nvedit.o)
 .debug_frame   0x0000143c       0x98 common/libcommon.a(command.o)
 .debug_frame   0x000014d4      0x214 common/libcommon.a(console.o)
 .debug_frame   0x000016e8       0x5c common/libcommon.a(devices.o)
 .debug_frame   0x00001744      0x13c common/libcommon.a(dlmalloc.o)
 .debug_frame   0x00001880       0x7c common/libcommon.a(env_common.o)
 .debug_frame   0x000018fc       0x68 common/libcommon.a(env_flash.o)
 .debug_frame   0x00001964       0x48 common/libcommon.a(exports.o)
 .debug_frame   0x000019ac       0x88 common/libcommon.a(flash.o)
 .debug_frame   0x00001a34      0x134 common/libcommon.a(lists.o)
 .debug_frame   0x00001b68       0x64 common/libcommon.a(s_record.o)
 .debug_frame   0x00001bcc      0x128 common/libcommon.a(xyzModem.o)
 .debug_frame   0x00001cf4       0x20 common/libcommon.a(crc16.o)
 .debug_frame   0x00001d14       0x28 lib_generic/libgeneric.a(crc32.o)
 .debug_frame   0x00001d3c       0x48 lib_generic/libgeneric.a(display_options.o)
 .debug_frame   0x00001d84      0x1dc lib_generic/libgeneric.a(string.o)
 .debug_frame   0x00001f60       0xe8 lib_generic/libgeneric.a(vsprintf.o)
 .debug_frame   0x00002048      0x1f4 lib_generic/libgeneric.a(zlib.o)
 .debug_frame   0x0000223c       0x38 board/ami/libami.a(ami.o)
 .debug_frame   0x00002274       0xd4 board/ami/libami.a(flash.o)
 .debug_frame   0x00002348      0x114 cpu/arm920t/libarm920t.a(cpu.o)
 .debug_frame   0x0000245c       0x88 cpu/arm920t/s3c24x0/libs3c24x0.a(serial.o)
 .debug_frame   0x000024e4       0x38 lib_arm/libarm.a(armlinux.o)
 .debug_frame   0x0000251c       0x20 lib_arm/libarm.a(cache.o)
 .debug_frame   0x0000253c       0x6c rtc/librtc.a(date.o)
 .debug_frame   0x000025a8       0x94 rtc/librtc.a(s3c24x0_rtc.o)

.debug_pubnames
                0x00000000     0x1d87
 .debug_pubnames
                0x00000000       0xdf cpu/arm920t/libarm920t.a(interrupts.o)
 .debug_pubnames
                0x000000df       0xd7 cpu/arm920t/s3c24x0/libs3c24x0.a(interrupts.o)
 .debug_pubnames
                0x000001b6       0x46 cpu/arm920t/s3c24x0/libs3c24x0.a(speed.o)
 .debug_pubnames
                0x000001fc       0x71 lib_arm/libarm.a(board.o)
 .debug_pubnames
                0x0000026d       0x1d lib_arm/libarm.a(div0.o)
 .debug_pubnames
                0x0000028a      0x3d7 net/libnet.a(net.o)
 .debug_pubnames
                0x00000661       0x20 net/libnet.a(tftp.o)
 .debug_pubnames
                0x00000681       0x3c net/libnet.a(bootp.o)
 .debug_pubnames
                0x000006bd       0x2e net/libnet.a(rarp.o)
 .debug_pubnames
                0x000006eb       0x25 net/libnet.a(eth.o)
 .debug_pubnames
                0x00000710       0x1f net/libnet.a(nfs.o)
 .debug_pubnames
                0x0000072f       0x8b drivers/libdrivers.a(cs8900.o)
 .debug_pubnames
                0x000007ba       0x5b common/libcommon.a(main.o)
 .debug_pubnames
                0x00000815       0x4c common/libcommon.a(cmd_autoscript.o)
 .debug_pubnames
                0x00000861       0x38 common/libcommon.a(cmd_bdinfo.o)
 .debug_pubnames
                0x00000899       0x47 common/libcommon.a(cmd_boot.o)
 .debug_pubnames
                0x000008e0       0xe4 common/libcommon.a(cmd_bootm.o)
 .debug_pubnames
                0x000009c4       0x5e common/libcommon.a(cmd_cache.o)
 .debug_pubnames
                0x00000a22       0x3a common/libcommon.a(cmd_console.o)
 .debug_pubnames
                0x00000a5c       0x4d common/libcommon.a(cmd_date.o)
 .debug_pubnames
                0x00000aa9       0x87 common/libcommon.a(cmd_elf.o)
 .debug_pubnames
                0x00000b30       0xb2 common/libcommon.a(cmd_flash.o)
 .debug_pubnames
                0x00000be2       0x53 common/libcommon.a(cmd_itest.o)
 .debug_pubnames
                0x00000c35      0x1c9 common/libcommon.a(cmd_load.o)
 .debug_pubnames
                0x00000dfe      0x1e7 common/libcommon.a(cmd_mem.o)
 .debug_pubnames
                0x00000fe5       0x36 common/libcommon.a(cmd_misc.o)
 .debug_pubnames
                0x0000101b       0xa4 common/libcommon.a(cmd_net.o)
 .debug_pubnames
                0x000010bf       0xd1 common/libcommon.a(cmd_nvedit.o)
 .debug_pubnames
                0x00001190       0xaa common/libcommon.a(command.o)
 .debug_pubnames
                0x0000123a      0x10e common/libcommon.a(console.o)
 .debug_pubnames
                0x00001348       0x76 common/libcommon.a(devices.o)
 .debug_pubnames
                0x000013be       0xb3 common/libcommon.a(dlmalloc.o)
 .debug_pubnames
                0x00001471       0x88 common/libcommon.a(env_common.o)
 .debug_pubnames
                0x000014f9       0x75 common/libcommon.a(env_flash.o)
 .debug_pubnames
                0x0000156e       0x35 common/libcommon.a(exports.o)
 .debug_pubnames
                0x000015a3       0x53 common/libcommon.a(flash.o)
 .debug_pubnames
                0x000015f6      0x116 common/libcommon.a(lists.o)
 .debug_pubnames
                0x0000170c       0x22 common/libcommon.a(s_record.o)
 .debug_pubnames
                0x0000172e       0xd5 common/libcommon.a(xyzModem.o)
 .debug_pubnames
                0x00001803       0x20 common/libcommon.a(crc16.o)
 .debug_pubnames
                0x00001823       0x1c lib_generic/libgeneric.a(crc32.o)
 .debug_pubnames
                0x0000183f       0x35 lib_generic/libgeneric.a(display_options.o)
 .debug_pubnames
                0x00001874      0x130 lib_generic/libgeneric.a(string.o)
 .debug_pubnames
                0x000019a4       0x5a lib_generic/libgeneric.a(vsprintf.o)
 .debug_pubnames
                0x000019fe       0xab lib_generic/libgeneric.a(zlib.o)
 .debug_pubnames
                0x00001aa9       0x1d lib_generic/libgeneric.a(ctype.o)
 .debug_pubnames
                0x00001ac6       0x2f board/ami/libami.a(ami.o)
 .debug_pubnames
                0x00001af5       0xb4 board/ami/libami.a(flash.o)
 .debug_pubnames
                0x00001ba9       0xb3 cpu/arm920t/libarm920t.a(cpu.o)
 .debug_pubnames
                0x00001c5c       0x74 cpu/arm920t/s3c24x0/libs3c24x0.a(serial.o)
 .debug_pubnames
                0x00001cd0       0x25 lib_arm/libarm.a(armlinux.o)
 .debug_pubnames
                0x00001cf5       0x22 lib_arm/libarm.a(cache.o)
 .debug_pubnames
                0x00001d17       0x38 rtc/librtc.a(date.o)
 .debug_pubnames
                0x00001d4f       0x38 rtc/librtc.a(s3c24x0_rtc.o)

.debug_aranges  0x00000000      0x6a0
 .debug_aranges
                0x00000000       0x20 cpu/arm920t/libarm920t.a(interrupts.o)
 .debug_aranges
                0x00000020       0x20 cpu/arm920t/s3c24x0/libs3c24x0.a(interrupts.o)
 .debug_aranges
                0x00000040       0x20 cpu/arm920t/s3c24x0/libs3c24x0.a(speed.o)
 .debug_aranges
                0x00000060       0x20 lib_arm/libarm.a(board.o)
 .debug_aranges
                0x00000080       0x20 lib_arm/libarm.a(div0.o)
 .debug_aranges
                0x000000a0       0x20 net/libnet.a(net.o)
 .debug_aranges
                0x000000c0       0x20 net/libnet.a(tftp.o)
 .debug_aranges
                0x000000e0       0x20 net/libnet.a(bootp.o)
 .debug_aranges
                0x00000100       0x20 net/libnet.a(rarp.o)
 .debug_aranges
                0x00000120       0x20 net/libnet.a(eth.o)
 .debug_aranges
                0x00000140       0x20 net/libnet.a(nfs.o)
 .debug_aranges
                0x00000160       0x20 drivers/libdrivers.a(cs8900.o)
 .debug_aranges
                0x00000180       0x20 common/libcommon.a(main.o)
 .debug_aranges
                0x000001a0       0x20 common/libcommon.a(cmd_autoscript.o)
 .debug_aranges
                0x000001c0       0x20 common/libcommon.a(cmd_bdinfo.o)
 .debug_aranges
                0x000001e0       0x20 common/libcommon.a(cmd_boot.o)
 .debug_aranges
                0x00000200       0x20 common/libcommon.a(cmd_bootm.o)
 .debug_aranges
                0x00000220       0x20 common/libcommon.a(cmd_cache.o)
 .debug_aranges
                0x00000240       0x20 common/libcommon.a(cmd_console.o)
 .debug_aranges
                0x00000260       0x20 common/libcommon.a(cmd_date.o)
 .debug_aranges
                0x00000280       0x20 common/libcommon.a(cmd_elf.o)
 .debug_aranges
                0x000002a0       0x20 common/libcommon.a(cmd_flash.o)
 .debug_aranges
                0x000002c0       0x20 common/libcommon.a(cmd_itest.o)
 .debug_aranges
                0x000002e0       0x20 common/libcommon.a(cmd_load.o)
 .debug_aranges
                0x00000300       0x20 common/libcommon.a(cmd_mem.o)
 .debug_aranges
                0x00000320       0x20 common/libcommon.a(cmd_misc.o)
 .debug_aranges
                0x00000340       0x20 common/libcommon.a(cmd_net.o)
 .debug_aranges
                0x00000360       0x20 common/libcommon.a(cmd_nvedit.o)
 .debug_aranges
                0x00000380       0x20 common/libcommon.a(command.o)
 .debug_aranges
                0x000003a0       0x20 common/libcommon.a(console.o)
 .debug_aranges
                0x000003c0       0x20 common/libcommon.a(devices.o)
 .debug_aranges
                0x000003e0       0x20 common/libcommon.a(dlmalloc.o)
 .debug_aranges
                0x00000400       0x20 common/libcommon.a(env_common.o)
 .debug_aranges
                0x00000420       0x20 common/libcommon.a(env_flash.o)
 .debug_aranges
                0x00000440       0x20 common/libcommon.a(exports.o)
 .debug_aranges
                0x00000460       0x20 common/libcommon.a(flash.o)
 .debug_aranges
                0x00000480       0x20 common/libcommon.a(lists.o)
 .debug_aranges
                0x000004a0       0x20 common/libcommon.a(s_record.o)
 .debug_aranges
                0x000004c0       0x20 common/libcommon.a(xyzModem.o)
 .debug_aranges
                0x000004e0       0x20 common/libcommon.a(crc16.o)
 .debug_aranges
                0x00000500       0x20 lib_generic/libgeneric.a(crc32.o)
 .debug_aranges
                0x00000520       0x20 lib_generic/libgeneric.a(display_options.o)
 .debug_aranges
                0x00000540       0x20 lib_generic/libgeneric.a(string.o)
 .debug_aranges
                0x00000560       0x20 lib_generic/libgeneric.a(vsprintf.o)
 .debug_aranges
                0x00000580       0x20 lib_generic/libgeneric.a(zlib.o)
 .debug_aranges
                0x000005a0       0x20 board/ami/libami.a(ami.o)
 .debug_aranges
                0x000005c0       0x20 board/ami/libami.a(flash.o)
 .debug_aranges
                0x000005e0       0x20 cpu/arm920t/libarm920t.a(cpu.o)
 .debug_aranges
                0x00000600       0x20 cpu/arm920t/s3c24x0/libs3c24x0.a(serial.o)
 .debug_aranges
                0x00000620       0x20 lib_arm/libarm.a(armlinux.o)
 .debug_aranges
                0x00000640       0x20 lib_arm/libarm.a(cache.o)
 .debug_aranges
                0x00000660       0x20 rtc/librtc.a(date.o)
 .debug_aranges
                0x00000680       0x20 rtc/librtc.a(s3c24x0_rtc.o)

.debug_str      0x00000000     0x3878
 .debug_str     0x00000000      0x14c cpu/arm920t/libarm920t.a(interrupts.o)
                                0x190 (size before relaxing)
 .debug_str     0x0000014c      0x1a0 cpu/arm920t/s3c24x0/libs3c24x0.a(interrupts.o)
                                0x262 (size before relaxing)
 .debug_str     0x000002ec       0xa1 cpu/arm920t/s3c24x0/libs3c24x0.a(speed.o)
                                0x16f (size before relaxing)
 .debug_str     0x0000038d      0x20e lib_arm/libarm.a(board.o)
                                0x2cd (size before relaxing)
 .debug_str     0x0000059b        0xe lib_arm/libarm.a(div0.o)
                                 0x3f (size before relaxing)
 .debug_str     0x000005a9      0x5a5 net/libnet.a(net.o)
                                0x76e (size before relaxing)
 .debug_str     0x00000b4e       0xec net/libnet.a(tftp.o)
                                0x26c (size before relaxing)
 .debug_str     0x00000c3a      0x176 net/libnet.a(bootp.o)
                                0x36a (size before relaxing)
 .debug_str     0x00000db0       0x4c net/libnet.a(rarp.o)
                                0x188 (size before relaxing)
 .debug_str     0x00000dfc       0x15 net/libnet.a(eth.o)
                                0x142 (size before relaxing)
 .debug_str     0x00000e11      0x26b net/libnet.a(nfs.o)
                                0x451 (size before relaxing)
 .debug_str     0x0000107c       0xf2 drivers/libdrivers.a(cs8900.o)
                                0x241 (size before relaxing)
 .debug_str     0x0000116e      0x166 common/libcommon.a(main.o)
                                0x22d (size before relaxing)
 .debug_str     0x000012d4       0xc7 common/libcommon.a(cmd_autoscript.o)
                                0x214 (size before relaxing)
 .debug_str     0x0000139b       0x35 common/libcommon.a(cmd_bdinfo.o)
                                0x209 (size before relaxing)
 .debug_str     0x000013d0       0x34 common/libcommon.a(cmd_boot.o)
                                0x145 (size before relaxing)
 .debug_str     0x00001404      0x2b8 common/libcommon.a(cmd_bootm.o)
                                0x5a9 (size before relaxing)
 .debug_str     0x000016bc       0x4f common/libcommon.a(cmd_cache.o)
                                0x14f (size before relaxing)
 .debug_str     0x0000170b       0xca common/libcommon.a(cmd_console.o)
                                0x1e4 (size before relaxing)
 .debug_str     0x000017d5       0x52 common/libcommon.a(cmd_date.o)
                                0x27a (size before relaxing)
 .debug_str     0x00001827      0x1ac common/libcommon.a(cmd_elf.o)
                                0x2f2 (size before relaxing)
 .debug_str     0x000019d3      0x14d common/libcommon.a(cmd_flash.o)
                                0x2c2 (size before relaxing)
 .debug_str     0x00001b20       0x90 common/libcommon.a(cmd_itest.o)
                                0x1a0 (size before relaxing)
 .debug_str     0x00001bb0      0x322 common/libcommon.a(cmd_load.o)
                                0x581 (size before relaxing)
 .debug_str     0x00001ed2      0x224 common/libcommon.a(cmd_mem.o)
                                0x379 (size before relaxing)
 .debug_str     0x000020f6       0x27 common/libcommon.a(cmd_misc.o)
                                0x139 (size before relaxing)
 .debug_str     0x0000211d       0x9e common/libcommon.a(cmd_net.o)
                                0x27b (size before relaxing)
 .debug_str     0x000021bb       0xe3 common/libcommon.a(cmd_nvedit.o)
                                0x303 (size before relaxing)
 .debug_str     0x0000229e       0xd1 common/libcommon.a(command.o)
                                0x1ee (size before relaxing)
 .debug_str     0x0000236f       0xee common/libcommon.a(console.o)
                                0x371 (size before relaxing)
 .debug_str     0x0000245d       0x44 common/libcommon.a(devices.o)
                                0x27b (size before relaxing)
 .debug_str     0x000024a1      0x2ac common/libcommon.a(dlmalloc.o)
                                0x496 (size before relaxing)
 .debug_str     0x0000274d       0x7e common/libcommon.a(env_common.o)
                                0x21e (size before relaxing)
 .debug_str     0x000027cb       0x5f common/libcommon.a(env_flash.o)
                                0x239 (size before relaxing)
 .debug_str     0x0000282a       0x25 common/libcommon.a(exports.o)
                                0x1ad (size before relaxing)
 .debug_str     0x0000284f       0x46 common/libcommon.a(flash.o)
                                0x17d (size before relaxing)
 .debug_str     0x00002895      0x1dc common/libcommon.a(lists.o)
                                0x308 (size before relaxing)
 .debug_str     0x00002a71       0x3a common/libcommon.a(s_record.o)
                                0x10a (size before relaxing)
 .debug_str     0x00002aab      0x1bd common/libcommon.a(xyzModem.o)
                                0x2cb (size before relaxing)
 .debug_str     0x00002c68       0x1c common/libcommon.a(crc16.o)
                                 0xe5 (size before relaxing)
 .debug_str     0x00002c84       0x3d lib_generic/libgeneric.a(crc32.o)
                                 0xee (size before relaxing)
 .debug_str     0x00002cc1       0x2d lib_generic/libgeneric.a(display_options.o)
                                0x100 (size before relaxing)
 .debug_str     0x00002cee       0xd0 lib_generic/libgeneric.a(string.o)
                                0x1c8 (size before relaxing)
 .debug_str     0x00002dbe       0x79 lib_generic/libgeneric.a(vsprintf.o)
                                0x196 (size before relaxing)
 .debug_str     0x00002e37      0x3c5 lib_generic/libgeneric.a(zlib.o)
                                0x5a8 (size before relaxing)
 .debug_str     0x000031fc        0x8 lib_generic/libgeneric.a(ctype.o)
                                 0x5a (size before relaxing)
 .debug_str     0x00003204      0x1b6 board/ami/libami.a(ami.o)
                                0x389 (size before relaxing)
 .debug_str     0x000033ba       0xef board/ami/libami.a(flash.o)
                                0x276 (size before relaxing)
 .debug_str     0x000034a9       0xa5 cpu/arm920t/libarm920t.a(cpu.o)
                                0x1b6 (size before relaxing)
 .debug_str     0x0000354e       0xfb cpu/arm920t/s3c24x0/libs3c24x0.a(serial.o)
                                0x294 (size before relaxing)
 .debug_str     0x00003649       0x46 lib_arm/libarm.a(armlinux.o)
                                0x2e2 (size before relaxing)
 .debug_str     0x0000368f       0x1a lib_arm/libarm.a(cache.o)
                                 0xd7 (size before relaxing)
 .debug_str     0x000036a9       0x62 rtc/librtc.a(date.o)
                                0x157 (size before relaxing)
 .debug_str     0x0000370b      0x16d rtc/librtc.a(s3c24x0_rtc.o)
                                0x2af (size before relaxing)

.comment        0x00000000      0x3cc
 .comment       0x00000000       0x12 cpu/arm920t/libarm920t.a(interrupts.o)
 .comment       0x00000012       0x12 cpu/arm920t/s3c24x0/libs3c24x0.a(interrupts.o)
 .comment       0x00000024       0x12 cpu/arm920t/s3c24x0/libs3c24x0.a(speed.o)
 .comment       0x00000036       0x12 lib_arm/libarm.a(board.o)
 .comment       0x00000048       0x12 lib_arm/libarm.a(div0.o)
 .comment       0x0000005a       0x12 net/libnet.a(net.o)
 .comment       0x0000006c       0x12 net/libnet.a(tftp.o)
 .comment       0x0000007e       0x12 net/libnet.a(bootp.o)
 .comment       0x00000090       0x12 net/libnet.a(rarp.o)
 .comment       0x000000a2       0x12 net/libnet.a(eth.o)
 .comment       0x000000b4       0x12 net/libnet.a(nfs.o)
 .comment       0x000000c6       0x12 drivers/libdrivers.a(cs8900.o)
 .comment       0x000000d8       0x12 common/libcommon.a(main.o)
 .comment       0x000000ea       0x12 common/libcommon.a(cmd_autoscript.o)
 .comment       0x000000fc       0x12 common/libcommon.a(cmd_bdinfo.o)
 .comment       0x0000010e       0x12 common/libcommon.a(cmd_boot.o)
 .comment       0x00000120       0x12 common/libcommon.a(cmd_bootm.o)
 .comment       0x00000132       0x12 common/libcommon.a(cmd_cache.o)
 .comment       0x00000144       0x12 common/libcommon.a(cmd_console.o)
 .comment       0x00000156       0x12 common/libcommon.a(cmd_date.o)
 .comment       0x00000168       0x12 common/libcommon.a(cmd_elf.o)
 .comment       0x0000017a       0x12 common/libcommon.a(cmd_flash.o)
 .comment       0x0000018c       0x12 common/libcommon.a(cmd_itest.o)
 .comment       0x0000019e       0x12 common/libcommon.a(cmd_load.o)
 .comment       0x000001b0       0x12 common/libcommon.a(cmd_mem.o)
 .comment       0x000001c2       0x12 common/libcommon.a(cmd_misc.o)
 .comment       0x000001d4       0x12 common/libcommon.a(cmd_net.o)
 .comment       0x000001e6       0x12 common/libcommon.a(cmd_nvedit.o)
 .comment       0x000001f8       0x12 common/libcommon.a(command.o)
 .comment       0x0000020a       0x12 common/libcommon.a(console.o)
 .comment       0x0000021c       0x12 common/libcommon.a(devices.o)
 .comment       0x0000022e       0x12 common/libcommon.a(dlmalloc.o)
 .comment       0x00000240       0x12 common/libcommon.a(env_common.o)
 .comment       0x00000252       0x12 common/libcommon.a(env_flash.o)
 .comment       0x00000264       0x12 common/libcommon.a(exports.o)
 .comment       0x00000276       0x12 common/libcommon.a(flash.o)
 .comment       0x00000288       0x12 common/libcommon.a(lists.o)
 .comment       0x0000029a       0x12 common/libcommon.a(s_record.o)
 .comment       0x000002ac       0x12 common/libcommon.a(xyzModem.o)
 .comment       0x000002be       0x12 common/libcommon.a(crc16.o)
 .comment       0x000002d0       0x12 lib_generic/libgeneric.a(crc32.o)
 .comment       0x000002e2       0x12 lib_generic/libgeneric.a(display_options.o)
 .comment       0x000002f4       0x12 lib_generic/libgeneric.a(string.o)
 .comment       0x00000306       0x12 lib_generic/libgeneric.a(vsprintf.o)
 .comment       0x00000318       0x12 lib_generic/libgeneric.a(zlib.o)
 .comment       0x0000032a       0x12 lib_generic/libgeneric.a(ctype.o)
 .comment       0x0000033c       0x12 board/ami/libami.a(ami.o)
 .comment       0x0000034e       0x12 board/ami/libami.a(flash.o)
 .comment       0x00000360       0x12 cpu/arm920t/libarm920t.a(cpu.o)
 .comment       0x00000372       0x12 cpu/arm920t/s3c24x0/libs3c24x0.a(serial.o)
 .comment       0x00000384       0x12 lib_arm/libarm.a(armlinux.o)
 .comment       0x00000396       0x12 lib_arm/libarm.a(cache.o)
 .comment       0x000003a8       0x12 rtc/librtc.a(date.o)
 .comment       0x000003ba       0x12 rtc/librtc.a(s3c24x0_rtc.o)

.debug_ranges   0x00000000      0x590
 .debug_ranges  0x00000000       0x38 cpu/arm920t/s3c24x0/libs3c24x0.a(interrupts.o)
 .debug_ranges  0x00000038       0x18 lib_arm/libarm.a(board.o)
 .debug_ranges  0x00000050       0xa0 net/libnet.a(net.o)
 .debug_ranges  0x000000f0       0x20 net/libnet.a(tftp.o)
 .debug_ranges  0x00000110       0x30 net/libnet.a(bootp.o)
 .debug_ranges  0x00000140       0x40 net/libnet.a(nfs.o)
 .debug_ranges  0x00000180       0x20 drivers/libdrivers.a(cs8900.o)
 .debug_ranges  0x000001a0       0x50 common/libcommon.a(main.o)
 .debug_ranges  0x000001f0       0x18 common/libcommon.a(cmd_autoscript.o)
 .debug_ranges  0x00000208       0x18 common/libcommon.a(cmd_flash.o)
 .debug_ranges  0x00000220       0x18 common/libcommon.a(cmd_itest.o)
 .debug_ranges  0x00000238       0x30 common/libcommon.a(cmd_load.o)
 .debug_ranges  0x00000268       0x30 common/libcommon.a(cmd_mem.o)
 .debug_ranges  0x00000298       0x18 common/libcommon.a(cmd_nvedit.o)
 .debug_ranges  0x000002b0       0x38 common/libcommon.a(command.o)
 .debug_ranges  0x000002e8       0x38 common/libcommon.a(console.o)
 .debug_ranges  0x00000320       0x18 common/libcommon.a(devices.o)
 .debug_ranges  0x00000338       0x50 common/libcommon.a(dlmalloc.o)
 .debug_ranges  0x00000388       0x50 common/libcommon.a(flash.o)
 .debug_ranges  0x000003d8       0x18 common/libcommon.a(xyzModem.o)
 .debug_ranges  0x000003f0       0x18 lib_generic/libgeneric.a(vsprintf.o)
 .debug_ranges  0x00000408      0x108 lib_generic/libgeneric.a(zlib.o)
 .debug_ranges  0x00000510       0x48 board/ami/libami.a(flash.o)
 .debug_ranges  0x00000558       0x38 rtc/librtc.a(s3c24x0_rtc.o)
